:10F800000C94387C0C94557C0C94557C0C94557C51
:10F810000C94557C0C94557C0C94557C0C94557C24
:10F820000C94557C0C94557C0C94557C0C94557C14
:10F830000C94557C0C94557C0C94557C0C94557C04
:10F840000C94557C0C94557C0C94557C0C94557CF4
:10F850000C94557C0C94557C0C94557C0C94557CE4
:10F860000C94557C0C94557C0C94557C0C94557CD4
:10F8700011241FBECFEFD0E1DEBFCDBF11E0A0E06D
:10F88000B1E0E6E4FCEF02C005900D92A630B107AE
:10F89000D9F711E0A6E0B1E001C01D92AC30B1078C
:10F8A000E1F70E94727C0C94217E0C94007C982FCE
:10F8B0008091C00085FFFCCF9093C6000895809191
:10F8C000C00087FFFCCF8091C600089588B1807C7E
:10F8D00088B981E085BF15BEE0910601F09107016E
:10F8E000099508952F923F924F925F926F927F9267
:10F8F0008F929F92AF92BF92CF92DF92EF92FF9240
:10F900000F931F93CF93DF9304B603FE06C0E091DD
:10F910000601F0910701099508C088E10FB6F89437
:10F9200080936000109260000FBE1092C50084E1C9
:10F930008093C40086E08093C20088E18093C10078
:10F9400082E60E94577C87B18F7387B926B186B152
:10F9500090E08078907030E020743070822B932B90
:10F960008034910529F081E60E94577C0E94667CD4
:10F9700080E70E94577C0E945F7C863509F477C03F
:10F980008735C8F48C3409F40CC18D3450F48234BA
:10F9900009F482C0853409F471C0813409F04FC183
:10F9A00028C0833509F45AC0843509F44AC080352B
:10F9B00009F045C1F6C0853669F1863648F48136CE
:10F9C000B1F0823609F460C0883509F038C156C0FC
:10F9D000803709F451C0813720F4873609F02FC1F0
:10F9E000E2C0833789F1843709F029C135C089E540
:10F9F000C0CF0E945F7C182F0E945F7C912E8824CC
:10FA000090E0882999299093090180930801880F33
:10FA1000991FA1C0E0E0F0E00BC007B600FCFDCFED
:10FA2000F999FECF23E020935700E895E050FF4F6F
:10FA300088EFE030F80788F3F0930B01E0930A01B8
:10FA4000B0C00E945F7CADC089E00E94577C86E90F
:10FA50000E94577C8EE18DCF82E01AC0C0E0D1E0D9
:10FA600003C00E94577C219688818823D1F780E3C8
:10FA70000E94577C82E37DCF83E57BCF8DE00E949F
:10FA8000577C0E94667C77CF89E50E94577C81E095
:10FA90000E94577C80E06DCF0E945F7C182F0E94EF
:10FAA0005F7C712E6624082F10E00629172991E04B
:10FAB0000130190708F0C3C00E945F7C863409F04A
:10FAC0004FC080910A0190910B018150984F18F01E
:10FAD00080E00E94577CA0900A01B0900B0107B60D
:10FAE00000FCFDCF6801D694C7947501C0E0D0E05A
:10FAF00016C00E945F7C082F0E945F7C582E442411
:10FB000010E00429152921E0F7010801209357008E
:10FB1000E895112482E090E0E80EF91E2196CC15BC
:10FB2000DD0538F3C601880F991F8A0D9B1D07B6A6
:10FB300000FCFDCFF999FECFE0910A01F0910B0195
:10FB400025E020935700E89507B600FCFDCFE1E1E2
:10FB5000E0935700E89590930B0180930A0121C030
:10FB6000853409F06CC0C0E0D0E018C00E945F7C12
:10FB70002091080130910901F999FECF1FBA32BDD9
:10FB800021BD80BD0FB6F894FA9AF99A0FBE2F5F87
:10FB90003F4F30930901209308012196C017D107E8
:10FBA00028F38DE0E6CE0E945F7C182F0E945F7CD8
:10FBB000312E2224E82EFF24E228F3280E945F7CC5
:10FBC0008634E9F4C0E0D0E016C0E0910A01F0917B
:10FBD0000B0105911491802F0E94577C812F0E9468
:10FBE000577C80910A0190910B01029690930B0132
:10FBF00080930A012296CE15DF0538F3BCCE8534FA
:10FC0000F1F410E016C08091080190910901F99972
:10FC1000FECF92BD81BDF89A80B50E94577C80913D
:10FC200008019091090101969093090180930801C0
:10FC30001F5F812F90E08E159F0528F39CCE8FE3E8
:06FC400098CEF894FFCFFE
:06FC460046444C2076004C
:040000030000F80001
:00000001FF
